:0200000480007A
:100000006F008004732F2034930F80006308FF0378
:10001000930F90006304FF03930FB0006300FF038E
:10002000130F000063040F0067000F00732F2034CC
:1000300063540F006F00400093E19153171F0000BD
:1000400023223FFC6FF09FFF93000000130100008C
:10005000930100001302000093020000130300004C
:100060009303000013040000930400001305000034
:10007000930500001306000093060000130700001C
:100080009307000013080000930800001309000004
:1000900093090000130A0000930A0000130B0000EC
:1000A000930B0000130C0000930C0000130D0000D4
:1000B000930D0000130E0000930E0000130F0000BC
:1000C000930F0000732540F16310050097020000B4
:1000D000938202017390523073500018970200000F
:1000E00093824202739052309B021000939252030B
:1000F0009382F2FF7390023B9302F0017390023AF5
:100100007350403097020000938242017390523046
:10011000735020307350303093010000970200007C
:10012000938282EE73905230130510001315F5017F
:10013000635C05000F00F00F930110009308D005D9
:10014000130500007300000093020000638A0200A0
:1001500073905210B7B200009B82921073902230BD
:100160007350003097020000938242017390123462
:10017000732540F173002030B78000009B8000E0C1
:100180003771DB061B0171DB1311C100130171DB39
:100190001311C100130171DB1311C100130171DBD5
:1001A00033872002B71300009B83032093010002D2
:1001B000631A7748B78000009B8000FC3771DB062C
:1001C0001B0171DB1311C100130171DB1311C1009D
:1001D000130171DB1311C100130171DB338720029E
:1001E000B71300009B83032493011002631C774420
:1001F00093000000130100003387200293030000E6
:100200009301200063107744930010001301100045
:100210003387200293031000930130006314774268
:1002200093003000130170003387200293035001C4
:100230009301400063187740930000003781FFFF6F
:10024000338720029303000093015000631C773E24
:10025000B7000080130100003387200293030000E1
:10026000930160006310773EB70000803781FFFF85
:10027000338720029B0310009393E30293017000E5
:100280006312773CB7B0AAFA9B80B0AA9390C000E3
:100290009380B0AA9390C0009380B0AA9390C000BE
:1002A0009380B0AA370103001B01D1E733872002F6
:1002B000B70301009B83F3F79301E00163147738E0
:1002C000B70003009B80D0E737B1AAFA1B01B1AA9F
:1002D0001311C1001301B1AA1311C1001301B1AA76
:1002E0001311C1001301B1AA33872002B703010023
:1002F0009B83F3F79301F001631677349300D000EA
:100300001301B000B38020029303F0089301800032
:10031000639A70329300E0001301B0003381200231
:100320009303A00993019000631E71309300D000E5
:10033000B38010029303900A9301A000639470307D
:10034000130200009300D0001301B0003387200295
:10035000130307001302120093022000E31452FE5D
:100360009303F0089301B000631E732C1302000086
:100370009300E0001301B000338720021300000057
:10038000130307001302120093022000E31252FE2F
:100390009303A0099301C0006316732A130200009F
:1003A0009300F0001301B000338720021300000017
:1003B0001300000013030700130212009302200031
:1003C000E31052FE9303500A9301D000631C73267E
:1003D000130200009300D0001301B0003387200205
:1003E0001302120093022000E31652FE9303F0085A
:1003F0009301E00063187724130200009300E000EB
:100400001301B00013000000338720021302120012
:1004100093022000E31452FE9303A0099301F0001D
:1004200063127722130200009300F0001301B00062
:100430001300000013000000338720021302120093
:1004400093022000E31252FE9303500A930100012D
:10045000631A771E130200009300D00013000000FF
:100460001301B00033872002130212009302200010
:10047000E31452FE9303F008930110016314771CF8
:10048000130200009300E000130000001301B0000D
:100490001300000033872002130212009302200091
:1004A000E31252FE9303A00993012001631C771805
:1004B000130200009300F00013000000130000007E
:1004C0001301B000338720021302120093022000B0
:1004D000E31252FE9303500A93013001631477161E
:1004E000130200001301B0009300D00033872002F4
:1004F0001302120093022000E31652FE9303F00849
:100500009301400163107714130200001301B0003F
:100510009300E00013000000338720021302120052
:1005200093022000E31452FE9303A00993015001AB
:10053000631A7710130200001301B0009300F0005B
:100540001300000013000000338720021302120082
:1005500093022000E31252FE9303500A93016001BC
:100560006312770E130200001301B00013000000A5
:100570009300D00033872002130212009302200060
:10058000E31452FE9303F00893017001631C770A91
:10059000130200001301B000130000009300E000FC
:1005A0001300000033872002130212009302200080
:1005B000E31252FE9303A0099301800163147708AC
:1005C000130200001301B00013000000130000002C
:1005D0009300F000338720021302120093022000E0
:1005E000E31252FE9303500A93019001631C7704B7
:1005F0009300F00133011002930300009301A00166
:10060000631271049300000233810002930300001F
:100610009301B00163187102B3000002930300005C
:100620009301C00163907002930010021301200235
:1006300033802002930300009301D0016314700003
:10064000631030020F00F00F6380010093911100DE
:1006500093E111009308D005138501007300000099
:100660000F00F00F930110009308D0051305000050
:0C06700073000000731000C000000000C8
:1010000000000000000000000000000000000000E0
:1010100000000000000000000000000000000000D0
:1010200000000000000000000000000000000000C0
:1010300000000000000000000000000000000000B0
:081040000000000000000000A8
:040000058000000077
:00000001FF
